:020000040800F2
:1000000000060020E1010008CD0D0008D10D000818
:10001000290E0008D10D0008FD0D0008E3010008BD
:10002000E3010008E3010008E30100083D210008A6
:10003000E3010008E3010008E3010008E301000810
:10004000E3010008E3010008E3010008E301000800
:10005000E3010008E30100081D32000849320008EE
:1000600075320008A1320008CD320008E301000813
:10007000E3010008E3010008E3010008E3010008D0
:10008000E3010008E3010008E3010008E3010008C0
:10009000E3010008E3010008E3010008F932000869
:1000A000E3010008E3010008E3010008E3010008A0
:1000B00091300008E3010008E3010008E3010008B3
:1000C000E3010008E3010008E3010008E301000880
:1000D000E3010008E3010008E3010008E301000870
:1000E00061330008E3010008E3010008E3010008B0
:1000F000E3010008E3010008E3010008E301000850
:10010000E3010008E3010008E3010008E30100083F
:10011000E3010008E3010008E3010008E30100082F
:10012000E3010008E3010008E3010008E30100081F
:10013000E3010008E3010008E3010008E30100080F
:10014000E3010008E3010008E3010008812800083A
:10015000E3010008E3010008E3010008E3010008EF
:10016000E3010008E3010008E3010008E3010008DF
:10017000E3010008E3010008E3010008E3010008CF
:10018000E3010008E3010008E3010008E3010008BF
:10019000E3010008E3010008E3010008E3010008AF
:1001A000E3010008E3010008E3010008E30100089F
:1001B000E3010008E3010008E3010008E30100088F
:1001C000E3010008E3010008E3010008E30100087F
:1001D000E3010008E3010008E3010008E30100086F
:1001E00002E000F000F8FEE772B6394880F30888B4
:1001F000384880F3098838484EF60851CEF200019D
:10020000086040F20000CCF200004EF63471CEF2ED
:1002100000010860BFF34F8FBFF36F8F40F2000003
:10022000C0F2F0004EF68851CEF200010860BFF334
:100230004F8FBFF36F8F4FF00000E1EE100A4EF6C4
:100240003C71CEF200010860062080F31488BFF3F1
:100250006F8F01F0D1FF02F077FE4FF055301F494C
:100260001B4A91423CBF41F8040BFAE71C49194A6A
:1002700091423CBF41F8040BFAE71A491A4A1B4B5A
:100280009A423EBF51F8040B42F8040BF8E70020F5
:100290001749184A91423CBF41F8040BFAE701F0B4
:1002A000AFFF02F0ADFE144C144DAC4203DA54F82B
:1002B000041B8847F9E700F041F8114C114DAC429E
:1002C00003DA54F8041B8847F9E701F097BF0000F0
:1002D000000600200022002000000008000000208E
:1002E0000006002090370008002200203C22002059
:1002F00040220020A42D0020E0010008E0010008B9
:10030000E0010008E00100082DE9F04F2DED108A12
:10031000C1F80CD0C3689D46BDEC108ABDE8F08FD3
:10032000002383F311882846A047002001F004FB36
:10033000FEE701F085FA00DFFEE7000038B501F0C6
:10034000CFFE044601F0F4FE0546D8B90F4B9C429F
:100350001AD001339C4218BF054641F2883404BFCD
:1003600001250024002001F0C5FE0DB100F058F871
:1003700000F000FD00F09EFB204600F0AFF800F01A
:100380004FF8F9E70024EDE70446EBE7010007B07A
:1003900008B500F061FBA0F120035842584108BDA8
:1003A00007B5054B02211B88ADF8043001A800F009
:1003B00071FB03B05DF804FB5C34000810B520232A
:1003C00083F311881248C3680BB101F051FB00237D
:1003D000104A0F484FF47A7101F0F8FA002383F3C2
:1003E00011880D4C236813B12368013B23606368B7
:1003F00013B16368013B6360084B1B7833B96368D2
:1004000023B9022000F02CFC3223636010BD00BF32
:1004100040220020BD0300085C230020542200205D
:1004200010B5254B254953F8042F013200D110BDDA
:100430008B42F8D1224C234B22689A423AD9224B64
:100440009B6803F1006303F540439A4232D20020D7
:1004500000F04AFB1D4B0220187000F0FFFB1C4B04
:100460001A6C00221A64196E1A66196E596C5A6455
:10047000596E5A665A6E5A6942F080025A615A6938
:1004800022F080025A615A691A6942F000521A61D8
:100490001A6922F000521A611B6972B60D4A0E4B9E
:1004A00013601B682268202181F311889D4683F325
:1004B0000888104710BD00BFFCBF00081CC0000822
:1004C00004C00008FFBF00080022002054220020C2
:1004D0000038024008ED00E000C000082DE9F04FB0
:1004E00099B0B94D00902022FF2110A8AC6800F00F
:1004F000E3FBB64A01951378A3B9B5480121C3605F
:100500001170202383F31188C3680BB101F0B0FA96
:100510000023B04AAE484FF47A7101F057FA002335
:1005200083F31188009BAC4A03B11360AB4B009D71
:10053000029300261E705660B2463746B14601202F
:1005400000F08CFB002D00F02582A34B1B68002BD4
:1005500040F0208219B0BDE8F08F0220FFF718FFAD
:10056000002840F01082009B002E08BF1D469C4BC7
:1005700002211B88ADF82C300BA800F08BFADEE7C7
:100580004FF47A7000F068FAB0F10008EBDB02205B
:10059000FFF7FEFE0028E6D008F1FF38B8F1040F9F
:1005A00000F2F381DFE808F0031E2124270018A8D9
:1005B000052340F8343D042100F06CFA012303FACE
:1005C00008F848EA0A0A5FFA8AFA4FF0000900F0D0
:1005D000C7FB27B10AF00B030B2B08BF0025FFF761
:1005E000DFFEACE704217848E6E704217D48E3E735
:1005F00004217D48E0E74FF01C09484600F076FAF8
:1006000009F104090B9004210BA800F043FAB9F199
:100610002C0FF2D1D2E7002FA5D00AF00B030B2B41
:10062000A1D10220FFF7B4FE804600289BD0012014
:100630006A4E00F059FA0220307000F00FFB0027DC
:100640005FFA87FB584600F05FFA054688B15846C6
:1006500000F06AFA01370028F2D146460025634BC4
:1006600002211B88ADF82C300BA800F013FA474686
:1006700065E701230220337000F0EEFA2C46019B5F
:100680009B689C4206D2204600F030FA0130E4D14B
:100690000434F4E7029B00241C704F4B46465C6018
:1006A0004746254693E7002F3FF45DAF0AF00B0362
:1006B0000B2B7FF458AF029B0220187000F0CEFA8B
:1006C000322000F0C9F9B0F1000BFFF64CAF1BF07F
:1006D00003087FF448AF019B996804EB0B028A4240
:1006E0003FF641AFBBF5807F3FF63DAF404A0392F6
:1006F000D8450FDA4FF47A7000F0AEF904900499FF
:100700000029FFF630AF039A049908F8021008F1A7
:100710000108ECE7C820FFF73BFE804600283FF4C5
:1007200022AF1F2C11D8C4F120075F4528BF5F46B8
:1007300010AB24F003003A462D49184400F092FA19
:100740003A46FF212A4800F0B7FA4FEAAB03DAB283
:1007500027490393204600F0B7FA074600283FF4E4
:100760007EAF039B04EB830431E70220FFF710FE0A
:1007700000283FF4F8AE00F0FDF900283FF4F3AE96
:100780004FF000084346019A9268904532D2B8F182
:100790001F0F12D8109A01320FD028F0030218A9A7
:1007A0000A4452F8202C0B92184604220BA900F0A0
:1007B0004FFB08F104080346E5E74046039300F0C9
:1007C00095F9039B0B90EFE70022002058230020AF
:1007D00040220020BD0300085C230020542200209A
:1007E0005E34000804220020082200206034000843
:1007F0005822002018A8042140F84C3D00F04AF986
:10080000E5E618A8002340F8343D642100F038F9EB
:1008100000287FF4A8AE0220FFF7BAFD00283FF4BD
:10082000A2AE0B9800F092F918AB43F8480D0421E2
:100830001846E3E718A8002340F8343D642100F08F
:100840001FF900287FF48FAE0220FFF7A1FD0028DA
:100850003FF489AE0B9800F087F918AB43F8440DCC
:10086000E5E70220FFF794FD00283FF47CAE00F09E
:1008700091F918AB43F8400DD9E70220FFF788FD46
:1008800000283FF470AE0BA9142000F089F98046CF
:1008900018A8042140F83C8D00F0FCF841460BA854
:1008A000ACE7322000F0D8F8B0F10008FFF65BAEFC
:1008B00018F0030F7FF457AE019A926808EB090312
:1008C00093423FF650AE0220FFF762FD00283FF44E
:1008D0004AAE28F00308C844C1453FF478AE484604
:1008E00000F004F904210A900AA800F0D3F809F1F5
:1008F0000409F1E74FF47A70FFF74AFD00283FF44E
:1009000032AE00F037F9002842D0109B01330BD0F3
:10091000082210A9002000F0D7F9002838D02022A2
:10092000FF2110A800F0C8F9FFF73AFD364801F0A2
:1009300009F80FE6002F3FF416AE0AF00B030B2B5D
:100940007FF411AE18A8002340F8343D642100F074
:1009500097F8804600287FF406AE0220FFF718FDC6
:1009600000283FF400AE0390FFF71AFD41F28830F3
:1009700000F0E8FF0B9800F027FA00F0F1F9039B74
:1009800045461F46DBE5074621E64FF00009EAE54C
:10099000B84664E6002000F05FF80490049B002B4A
:1009A000FFF6D0AD012000F057F9049B213B122B3C
:1009B0003FF6C5AD01A252F823F000BF5B05000869
:1009C00081050008170600083F0500083F050008DC
:1009D0003F050008A7060008A30800086B070008E9
:1009E0000308000835080008630800083F050008F0
:1009F0007B0800083F050008F5080008CF0500083F
:100A00003F05000835090008A086010070B50F4BAE
:100A10000C4619780131C9B2012906460FD80C4895
:100A200003681D6A4FF47A73534331462246A84740
:100A3000844204D1074B00221A70012070BD4FF48C
:100A4000FA7000F07FFF002070BD00BF0C22002074
:100A5000502500209023002007B502AB002203F8A8
:100A6000012D012102461846FFF7D0FF20B19DF865
:100A7000070003B05DF804FB4FF0FF30F9E700001A
:100A80000A4608B50421FFF7C1FF80F00100C0B29B
:100A9000404208BD30B4054C2368DD69044B0A466A
:100AA000AC460146204630BC604700BF50250020C0
:100AB000A086010070B501F017FA094C094E20809C
:100AC000002530682388834208D901F007FA33688B
:100AD00005440133B5F5404F3360F2D370BD00BF1C
:100AE000922300206423002001F0ACBA00F10060E2
:100AF00000F540400068704700F10060920000F58A
:100B0000404001F037BA0000054B1A68054B1B88BE
:100B10009B1A834202D9104401F0E0B900207047CB
:100B2000642300209223002038B5074D044628682E
:100B3000204401F0DBF928B928682044BDE838409A
:100B400001F0ECB938BD00BF6423002010F00303AE
:100B500008D1B0F5047F05D200F10050A0F508409F
:100B60000068704700207047014BC058704700BFB5
:100B7000107AFF1F064991F8243033B10023082270
:100B8000086A81F82430FFF7B7BF0120704700BF23
:100B900068230020014B1868704700BF002004E064
:100BA00070B52A4B1C68C4F30B03240C63B140F2EC
:100BB0001342934231D040F2194293422FD040F277
:100BC000214293422DD10323214A0C2505FB032307
:100BD0005D6893F9082042F201039C4224D0B4F5E9
:100BE000805F23D041F201039C4221D041F20303F4
:100BF0009C421FD041F207039C4208BF3122441E91
:100C00000C44013D0B46A3421ED215F9016F581C3E
:100C100096B1034600F8016CF5E70123D4E70223FF
:100C2000D2E73F220B4DD6E73322E3E74122E1E74B
:100C30005A22E4E75922E2E72C2584421D7001D9AB
:100C4000981C5A70401A70BD1846FBE7002004E05B
:100C500070340008643400087047000070470000DA
:100C60007047000010B50023934203D0CC5CC454FD
:100C70000133F9E710BD000030B5441E14F9010F2F
:100C80000B4660B193F90050854201F1010106D194
:100C90001AB993F90020801A30BD013AEEE7002A14
:100CA000F7D1104630BD000002460346981A13F9EA
:100CB000011B0029FAD1704702440346934202D037
:100CC00003F8011BFAE770472DE9F047234C94F82D
:100CD000243005468846174683BB2E46DFF87C90B5
:100CE000C7B394F824302BB92022FF21484626624E
:100CF000FFF7E2FF94F82400C0F10805BD4228BFC9
:100D00003D465FFA85FAAD0041462A4604EB800075
:100D1000FFF7A8FF94F82430A7EB0A079A445FFA7C
:100D20008AFABAF1080F2E44A844FFB284F824A02E
:100D3000D6D1FFF71FFF0028D2D108E0266A06EBC4
:100D40008306B042CAD0FFF715FF0028C5D10020A6
:100D5000BDE8F0870120BDE8F08700BF68230020D0
:100D6000024B1A78024B1A70704700BF9023002084
:100D70000C22002038B5104D104C284600F0F8F831
:100D80002146284600F020F924680D48626DD2F80B
:100D9000043843F00203C2F8043800F0D3FD0949D7
:100DA000204600F01DFA626DD2F8043823F00203E9
:100DB000C2F8043838BD00BF502500206435000853
:100DC00040420F008C35000870470000FEE700002D
:100DD00000B59BB0EFF3098168226846FFF742FF38
:100DE000EFF30583044B9A6BDA6A9A6A9A6A9A6AF5
:100DF0009A6A9A6A9B6AFEE700ED00E000B59BB034
:100E0000EFF3098168226846FFF72CFFEFF30583B3
:100E1000044B9A6B9A6A9A6A9A6A9A6A9A6A9B6A65
:100E2000FEE700BF00ED00E000B59BB0EFF30981E5
:100E300068226846FFF716FFEFF30583034B5A6BF2
:100E40009A6A9A6A9A6A9A6A9B6AFEE700ED00E0DB
:100E500030B5084D0A4491420BD011F8013B0924EA
:100E60005840013CF7D040F300032B4083EA500088
:100E7000F7E730BD2083B8ED026843681143016095
:100E800003B118477047000013B5446BD4F894348D
:100E90001A681178042915D1217C022912D11979F7
:100EA000128901238B4013420CD101A904F14C009B
:100EB00001F04EFFD4F89444019B2179024620684A
:100EC00000F0DAF902B010BD143001F0D1BE00001C
:100ED0004FF0FF33143001F0CBBE00004C3001F076
:100EE000A3BF00004FF0FF334C3001F09DBF000066
:100EF000143001F09FBE00004FF0FF31143001F0BC
:100F000099BE00004C3001F06FBF00004FF0FF327F
:100F10004C3001F069BF0000D0F8942438B5136854
:100F200019780429054601D0012038BD017C022929
:100F3000FAD112795C89012090400440F4D105F186
:100F4000140001F031FE02460028EDD0D5F894548B
:100F50004FF480732868697900F07CF9204638BD29
:100F6000406BFFF7D9BF00000020704770470000BA
:100F70007FB5124B0360002343608360C36001258B
:100F800002260F4B057404460290019300F184027F
:100F9000294600964FF48073143001F0E1FD094BAF
:100FA0000193029400964FF4807304F5237229464E
:100FB00004F14C0001F0A8FE04B070BDC03400087C
:100FC000610F0008890E00080B68202282F3118847
:100FD0000A7903EB820290614A79093243F82200D0
:100FE0008A7912B103EB8203986102230374C0F87B
:100FF0009414002383F311887047000038B5037FF1
:10100000044613B190F85430ABB9201D01250221DC
:10101000FFF732FF04F1140025776FF0010100F0B3
:10102000B9FC84F8545004F14C006FF00101BDE8A4
:10103000384000F0AFBC38BD10B501210446043083
:10104000FFF71AFF0023237784F8543010BD000007
:1010500038B504460025143001F09AFD04F14C0027
:10106000257701F069FE201D84F854500121FFF717
:1010700003FF2046BDE83840FFF74EBF90F84430EC
:1010800003F06003202B19D190F84520212A0AD0C3
:10109000222A4FF000030ED0202A0FD1084A826383
:1010A0000722C26304E0064B83630723C363002364
:1010B0000364012070478363C363F9E7002070472E
:1010C0000D220020D0F8943437B51A68117804291D
:1010D00004461AD1017C022917D1197912890123FA
:1010E0008B40134211D100F14C05284601F0E4FE7B
:1010F00058B101A9284601F02BFED4F89444019B75
:1011000021790246206800F0B7F803B030BD000036
:1011100000EB8103F7B59C6905460E46F4B1202328
:1011200083F3118805EB8607201D0821FFF7A4FE35
:10113000FB685B691B684C3413B1204601F016FE56
:1011400001A9204601F004FE024648B1019B314648
:10115000284600F091F8002383F3118803B0F0BD16
:10116000FB685A691268002AF5D01B8A013B1340BC
:10117000F1D105F14402EAE7093138B550F82140D0
:10118000DCB1202383F31188D4F8942413685279B6
:1011900003EB8203DB689B695D6845B1042160183D
:1011A000FFF76AFE294604F1140001F007FD20460E
:1011B000FFF7B2FE002383F3118838BD70470000AB
:1011C00001F0B0B80123037000234360C361836260
:1011D0000362C3624362036303814381704700007B
:1011E00038B50446202383F3118800254160C5608B
:1011F00005614561856101F0A5F80223237085F33F
:10120000118838BD70B500EB810305465069DA607E
:101210000E46144618B110220021FFF74DFDA069BB
:1012200018B110220021FFF747FD31462846BDE8DE
:10123000704001F051B90000028902F00102028100
:10124000428902F001024281002202614261826110
:1012500001F0D6B9F0B400EB81044789E4680125B8
:10126000A4698D403D43458123600023A2606360F3
:10127000F0BC01F0F1B90000F0B400EB8104078983
:10128000E468012564698D403D43058123600023A6
:10129000A2606360F0BC01F06BBA000070B502237D
:1012A000002504460370A0F84C5080F84E5080F89A
:1012B0004F5005814581C56005614561856180F8B4
:1012C000345001F0A5F863681B6823B12946204615
:1012D000BDE87040184770BD037880F85030052392
:1012E000037043681B6810B504460BB1042198478E
:1012F00000232381638110BD436890F850201B6850
:1013000002700BB1052118477047000090F8343087
:1013100070B5044613B1002380F8343004F1440260
:10132000204601F08FF963689B6863BB94F84450D2
:1013300015F0600615D194F8453005F07F0545EAB3
:10134000032540F202339D4200F00E815BD8022D4E
:1013500000F0DC803FD8002D00F08780012D00F0E8
:10136000CF800021204601F0C7FB0021204601F07C
:10137000B9FB63681B6813B1062120469847062312
:1013800084F8343070BD204698470028CED094F8B9
:101390004B2094F84A3043EA0223E26B934238BF71
:1013A000E36394F94430E56B002B4FF0200380F2A7
:1013B000FD80002D00F0EC80092284F8342083F3B6
:1013C00011880021E36BA26B2046FFF755FF002335
:1013D00083F3118870BDB5F5817F00F0B180B5F55C
:1013E000407F49D0B5F5807FBBD194F84630012BC2
:1013F000B7D1B4F84C3023F00203A4F84C30A66304
:10140000E6632664C3E740F201639D421ED8B5F54A
:10141000C06F3BD2B5F5A06FA3D1B4F84430B3F59B
:10142000A06F0ED194F8463084F84E30204601F07B
:1014300047F863681B6813B10121204698470323CE
:1014400023700023A363E3632364A0E7B5F5106F63
:1014500032D040F602439D4252D0B5F5006F80D1A4
:1014600004F14F03A363012324E004F14C03A363BD
:101470000223E36325648AE794F84630012B7FF466
:1014800070AFB4F84C3043F00203B6E794F849204B
:10149000616894F848304D6894F8471043EA022395
:1014A000204694F84620A84700283FF45AAF4368E6
:1014B000A3630368E363A4E72378042B10D12023FC
:1014C00083F311882046FFF7B7FE86F3118863681F
:1014D00084F84F601B68032121700BB120469847A8
:1014E00094F84630002BACD084F84F30042323709E
:1014F00063681B68002BA4D0022120469847A0E710
:10150000374BA3630223E36300239DE794F848105D
:1015100011F0800F204601F00F010ED001F084F889
:10152000012806D002287FF41CAF2E4BA363E06392
:1015300067E72D4BA363E56363E701F067F8EFE727
:1015400094F84630002B7FF40CAF94F8483013F039
:101550000F013FF476AF1A06204602D501F0E0FAFB
:101560006FE701F0D3FA6CE794F84630002B7FF474
:10157000F8AE94F8483013F00F013FF462AF1B0649
:10158000204602D501F0B8FA5BE701F0ABFA58E764
:10159000142284F8342083F311882B462A462946E6
:1015A0002046FFF757FE85F3118870BD5DB1152207
:1015B00084F8342083F311880021E36BA26B20466A
:1015C000FFF748FE03E70B2284F8342083F31188E9
:1015D0002B462A4629462046FFF74EFEE3E700BF8A
:1015E000F0340008E8340008EC34000838B590F80E
:1015F00034300446152B29D8DFE803F03E2828288C
:1016000028283E28280B293928282828282828284F
:101610003E3E90F84B1090F84A20C36B42EA0122FC
:101620009A4214D9C268128AB3FBF2F502FB15354F
:101630006DB9202383F311882B462A462946FFF7EC
:101640001BFE85F311880A2384F8343038BD142337
:1016500084F83430202383F3118800231A46194676
:101660002046FFF7F7FD002383F3118838BD036C94
:1016700003B198470023E7E7002101F03DFA00217C
:10168000204601F02FFA63681B6813B1062120463B
:1016900098470623D8E7000090F83420152A38B57B
:1016A000044622D80123934040F6416213421DD1E3
:1016B00013F480150FD19B0217D50B2380F834301B
:1016C000202383F311882B462A462946FFF7D4FDB1
:1016D00085F3118838BDC3689B695B682BB9036CBF
:1016E00003B19847002384F8343038BD002101F05D
:1016F00003FA0021204601F0F5F963681B6813B175
:101700000621204698470623EDE70000024B002201
:101710001B605B609A607047942300200023037471
:101720008268054B1B6899689142FBD25A68036036
:1017300042601060586070479423002008B5202351
:1017400083F31188037C032B05D0042B0DD02BB918
:1017500083F3118808BD436900221A604FF0FF33FC
:101760004361FFF7DBFF0023F2E790E80C001A600B
:1017700002685360F2E70000002303748268054B9F
:101780001B6899689142FBD85A68036042601060F8
:101790005860704794230020054B19690874186835
:1017A00002681A605360186101230374FEF7ACBD30
:1017B0009423002030B54B1C87B005460A4C10D04E
:1017C00023690A4A01A800F001F92846FFF7E4FF5F
:1017D000049B13B101A800F04BF92369586907B0C5
:1017E00030BDFFF7D9FFF8E7942300203D1700082C
:1017F00038B50C4D41612B6981689A689142044665
:1018000003D8BDE83840FFF789BF1846FFF7B4FF9B
:1018100001232C61014623742046BDE83840FEF7C1
:1018200073BD00BF94230020044B1A681B699068A5
:101830009B68984294BF00200120704794230020A9
:1018400010B5084C236820691A6822605460012290
:1018500023611A74FFF790FF01462069BDE810402C
:10186000FEF752BD94230020FEE7000010B50C4C9B
:10187000FFF74CFF00F09CF880220A49204600F058
:1018800021F8012344F8180C037400F067FC0023CE
:1018900083F3118862B60448BDE8104000F034B804
:1018A000BC230020F4340008FC34000800F01AB90E
:1018B000034B59685A68521A9042FBD8704700BFD0
:1018C000001000E08260022202740022427470471D
:1018D0008368A3F17C0243F80C2C026943F83C2C8A
:1018E000426943F8382C074A43F81C2CC26843F875
:1018F000102C022203F8082C002203F8072CA3F175
:10190000180070472103000810B5202383F31188C5
:10191000FFF7DEFF00210446FFF76AFF002383F391
:101920001188204610BD0000024B1B6958610F2032
:10193000FFF732BF94230020202383F31188FFF7A1
:10194000F3BF000008B50146202383F31188082067
:10195000FFF730FF002383F3118808BD49B1064B20
:1019600042681B6918605A60136043600420FFF7E7
:1019700021BF4FF0FF307047942300200368984246
:1019800006D01A680260506059611846FFF7C6BE5B
:101990007047000038B504460D462068844200D1E7
:1019A00038BD036823605C604561FFF7B7FEF4E76C
:1019B000054B03F114025A619A614FF0FF32DA616C
:1019C00000221A62704700BF94230020F8B5274F09
:1019D0000361C2600D46044601F0A2FA3B46022DA7
:1019E00053F8142F294638BF02219A423E461D461D
:1019F0000AD138627C61BC61084422606260A160E7
:101A0000BDE8F84001F07ABAD7F820E0A0EB0E0369
:101A10005F181FD300279068834217D8376AAA42FD
:101A20001F44376201D0C01A906073699A6891426E
:101A300019D85A682360626014605C60A16098687D
:101A4000411A99604FF0FF33F361F8BD97601B1A9C
:101A50001268E0E793689F4203D20EEB070001F0A3
:101A60005BFA3946E1E7891A1B68DFE79423002017
:101A700038B51B4B01685A6990421D4603F11402A8
:101A80000CD0446821600368002193425C60C1600F
:101A900025D09A6881680A449A6038BD59614A60C5
:101AA0005B6900219342C16003D1BDE8384001F079
:101AB0002DBA9A6881680A449A602C6A01F030FA5B
:101AC0006A699268001B824209D9111A012998BFDC
:101AD000821C286ABDE83840104401F01DBA38BDA8
:101AE000942300202DE9F84F204C0027656904F16C
:101AF0001406B84601F014FA236AA0EB030AAB6897
:101B000053451DD84FF02009236AAA68D5F80CB0B8
:101B100013442362AB68AAEB030A2B68B3425E60EE
:101B20006361EF6001D101F0F1F988F31188286950
:101B3000D84789F311886569AB689A45E4D2D9E73B
:101B40006369B34210D020629A68A2EB0A029A60DD
:101B5000226AAB68821A9B1A022B2CBFC018023073
:101B6000BDE8F84F01F0D8B9BDE8F88F9423002004
:101B700000207047FEE70000704700004FF0FF3084
:101B800070470000022906D0032906D00129064823
:101B900018BF0020704705487047032A9ABF0448C1
:101BA00000EBC20000207047E83500089C350008B3
:101BB0001C22002070B59AB001AD064608462946A1
:101BC000144600F0BDF82846FFF76EF8C0B2431C7B
:101BD0005B0086E81800237003236370002302343F
:101BE0001946DAB2904204F1020401D81AB070BD6D
:101BF000EA5C04F8022C04F8011C0133F1E7000050
:101C000008B5202383F311880348FFF75BFA00230C
:101C100083F3118808BD00BF5025002090F84430A0
:101C200003F01F02012A07D190F845200B2A03D1A7
:101C300000238363C36312E003F06003202B11D100
:101C4000B0F8483073B990F84520212A03D0222AF1
:101C5000EFD0202A06D1044A82630722C2630364BC
:101C600001207047FFF70ABA1422002010B504467D
:101C7000052916D8DFE801F016150316161D2023D6
:101C800083F311880E4A0121FFF7BCFA20460D4A62
:101C90000221FFF7B7FA0C48FFF7DAF9002383F3C4
:101CA000118810BD202383F311880748FFF7A6F998
:101CB000F4E7202383F311880348FFF7BDF9EDE72C
:101CC0001C350008403500085025002038B50C4D63
:101CD0000C4C0D492A4604F10800FFF76BFF05F193
:101CE000CA0204F110000949FFF764FF05F5CA7242
:101CF00004F118000649BDE83840FFF75BBF00BF9C
:101D0000182A00201C2200206C35000876350008B7
:101D10008135000870B5044608460D46FEF7C4FF3D
:101D2000C6B22046013403780BB9184670BD32465E
:101D30002946FEF7A1FF0028F3D1012070BD000065
:101D40002DE9F04704460D46FEF7AEFF2D49C6B219
:101D50002046FFF7DFFF08B10836F6B22A492046D1
:101D6000FFF7D8FF08B11036F6B2632E0BD8DFF8B4
:101D70009480DFF89490254FDFF89CA0267846B930
:101D80002E70BDE8F08721462846BDE8F04701F0F7
:101D90005DBB252E31D1072241462046FEF76CFF60
:101DA00080B91B4B2A4603F10C0153F8040B42F88F
:101DB000040B8B42F9D119889B78118093700734FA
:101DC0000F35DBE7082249462046FEF755FFA0B94C
:101DD000104BAA1C13F8011F09095345C95D02F8ED
:101DE000021C197801F00F0102F10202C95D02F82C
:101DF000031CEFD118350834C0E72E7001340135CB
:101E0000BCE700BF0836000881350008203600080E
:101E1000103600080F7AFF1F1B7AFF1FBFF34F8F8A
:101E2000024AD368DB03FCD4704700BF003C024089
:101E300008B5094B1B7873B9FFF7F0FF074B1A6918
:101E4000002ABFBF064A5A6002F188325A601A68F7
:101E500022F480621A6008BD762C0020003C02400B
:101E60002301674508B50B4B1B7893B9FFF7D6FFE5
:101E7000094B1A6942F000421A611A6842F4805212
:101E80001A601A6822F480521A601A6842F480625A
:101E90001A6008BD762C0020003C02400B2870B56B
:101EA00013D80B4A0B4C137863B90B4E4FF00061FB
:101EB00044F8231056F8235001330C2B2944F7D152
:101EC0000123137054F8200070BD002070BD00BFC6
:101ED000A82C0020782C002034360008014B53F841
:101EE00020007047343600080C2070470B2810B5CE
:101EF000044601D9002010BDFFF7D0FF064B53F870
:101F000024301844C21A0BB9012010BD12680132E6
:101F1000F0D1043BF6E700BF343600080B2810B5BB
:101F2000044621D8FFF77AFFFFF782FF0F4AF32319
:101F3000D360C300DBB243F4007343F002031361C8
:101F4000136943F480331361FFF768FFFFF7A6FFBF
:101F5000074B53F8241000F0DDF8FFF783FF20460D
:101F6000BDE81040FFF7C2BF002010BD003C02409A
:101F7000343600082DE9F84312F00103154640D12C
:101F80008218B2F1016F3CD22C4B1B6813F0010395
:101F900037D02B4CFFF74CFFF323E360FFF73EFFF6
:101FA00040F20127032D01D9830713D0244C0F469B
:101FB000401A40F20118EB1B0B44012B00EB070603
:101FC000236924D823F001032361FFF74BFF01208D
:101FD000BDE8F883236923F44073236123693B43FD
:101FE000236151F8046B0660BFF34F8FFFF716FFB4
:101FF00003689E4208D0236923F001032361FFF7A1
:1020000031FF0020BDE8F883043D0430CAE723F423
:1020100040732361236943EA08032361B94637F813
:10202000023B3380BFF34F8FFFF7F8FE3688B9F8D5
:102030000030B6B2B342BED0DDE700BF0038024088
:10204000003C0240084908B50B7828B153B9FFF7A6
:10205000EFFE01230B7008BD23B1BDE808400870F6
:10206000FFF700BF08BD00BF762C002010B502446A
:10207000064B0439D2B2904200D110BD441C00B2CC
:1020800053F8200041F8040FE0B2F4E75028004074
:10209000104B30B51C6F240407D41C6F44F400743B
:1020A0001C671C6F44F400441C670B4C236843F40A
:1020B000807323600244094B0439D2B2904200D1AC
:1020C00030BD441C00B251F8045F43F82050E0B228
:1020D000F4E700BF00380240007000405028004084
:1020E00007B5012201A90020FFF7C0FF019803B046
:1020F0005DF804FB13B50446FFF7F2FFA04206D0DB
:1021000002A9012241F8044D0020FFF7C1FF02B0EF
:1021100010BD000070470000034B1B689B0042BFCE
:10212000024B01221A70704774380240A92C00201B
:10213000014B1878704700BFA92C0020EFF30983EA
:1021400005494A6822F001024A60683383F309882E
:10215000002383F31188704730EF00E0202080F3E4
:10216000118862B60B4B0C4AD96821F4E06109046E
:10217000090C0A430949DA60CA6842F08072CA60F1
:1021800007490A6842F001020A601022DA7783F8F0
:102190002200704700ED00E00003FA05F0ED00E0DA
:1021A000001000E010B5202383F311880E4B5B680C
:1021B00013F4006314D0F1EE103AEFF30984683C95
:1021C0004FF08073E361094BDB68236684F3098871
:1021D000FFF72AFB10B1064BA36110BD054BFBE7CF
:1021E00083F3118810BD00BF00ED00E030EF00E088
:1021F000330300083603000870470000FEE70000C4
:10220000084A094B09498B4204D3094A00219342E9
:1022100005D3704752F8040F43F8040BF3E743F873
:10222000041BF4E7C8370008A42D0020A42D0020CB
:10223000A42D0020836D70B5446D9E6800214FF081
:10224000FF354A01A3180131D3F800090028BEBFA9
:10225000D3F8000940F08040C3F80009D3F8000B20
:102260000028BEBFD3F8000B40F08040C3F8000B3D
:10227000A3188E42C3F80859C3F8085BE1D24FF0A7
:102280000113C4F81C3870BD890141F020010161BF
:1022900003699B06FCD41220FFF70ABB204B03EB1B
:1022A00080022DE9F047D2F80CE05D6DDEF81420D5
:1022B000461CD2F800C005EB063605EB4018516805
:1022C00061450BD3D5F83428012303FA00F022EA44
:1022D0000000C5F834081846BDE8F087BEF8104085
:1022E000ACEB0103A34228BF2346D8F81849A4B297
:1022F000B3EB840F10D894681F46A4F1040959F871
:1023000004AFC6F800A0042F01D9043FF7E71C442E
:102310000B4494605360D2E70020BDE8F08700BF13
:10232000AC2C002010B5054C2046FEF74BFF4FF0BB
:10233000A0436365024BA36510BD00BFAC2C002019
:10234000883600080378012B70B5054650D12A4B1A
:10235000446D98421BD1294B5A6B42F080025A635C
:102360005A6D42F080025A655A6D5A6942F08002F5
:102370005A615A6922F080025A610E2143205B693A
:1023800000F0D8FB1E4BE3601E4BC4F8003800235E
:10239000C4F8003EC02323606E6D4FF40413A363A2
:1023A0003369002BFCDA012333610C20FFF780FA3C
:1023B0003369DB07FCD41220FFF77AFA3369002B6C
:1023C000FCDA0026A6602846FFF734FF6B68C4F8E5
:1023D0001068DB68C4F81468C4F81C684BB90A4B71
:1023E000A3614FF0FF336361A36843F00103A3606F
:1023F00070BD064BF4E700BFAC2C00200038024053
:102400004014004003002002003C30C0083C30C0B3
:10241000F8B5446D054600212046FFF735FFA96D4C
:1024200000234FF001128F68C4F834384FF0006673
:10243000C4F81C284FF0FF3004EB431201339F42D5
:10244000C2F80069C2F8006BC2F80809C2F8080BAC
:10245000F2D20B686A6DEB65636210231361166933
:1024600016F01006FBD11220FFF722FAD4F800383C
:1024700023F4FE63C4F80038A36943F4402343F017
:102480001003A3610923C4F81038C4F814380A4BA8
:10249000EB604FF0C043C4F8103B084BC4F8003B5E
:1024A000C4F81069C4F80039EB6D03F1100243F46D
:1024B0008013EA65A362F8BD64360008408000100E
:1024C000426D90F84E10D2F8003823F4FE6343EAD0
:1024D0000113C2F8003870472DE9F0410EB200EB4D
:1024E00086080D46D8F80C100F6807F00303022B7E
:1024F00050D0032B50D03D4A3D4F012B18BF1746FB
:10250000446D4FEA451E04EB0E030022C3F8102B66
:102510008A6905F1100C002A40D04A8A05F1580357
:102520005B013A43E2500123D4F81C2803FA0CF370
:102530001343A6444A69C4F81C380023CEF8103966
:1025400005F13F03002A39D00A8A898B92080129B4
:1025500088BF4A43C16D04EB8303561841EA024227
:10256000C66529465A602046FFF78EFED8F80C3023
:102570001B8A43EA85531F4305F148035B01E7507B
:102580000123D4F81C2803FA05F51543C4F81C5898
:10259000BDE8F081174FB3E7174FB1E704EB4613DF
:1025A000D3F8002B22F40042C3F8002BD4F81C28E7
:1025B000012303FA0CF322EA0303BAE704EB8303D3
:1025C0000E4A5A6004EB461629462046FFF75CFE89
:1025D000D6F8003923F40043C6F80039D4F81C3883
:1025E000012202FA05F523EA0505CFE70080001075
:1025F000008004100080081000800C10000400020D
:10260000826D1268C265FFF715BE00005831436D38
:1026100049015B5813F4004004D013F4001F14BFA9
:1026200001200220704700004831436D49015B588A
:1026300013F4004004D013F4001F14BF0120022043
:102640007047000000EB8101CB68196A0B681360CA
:102650004B6853607047000000EB810330B5DD68C4
:10266000AA691368D36019B9402B84BF4023136053
:102670006B8A1468426D1C44013CB4FBF3F4634361
:10268000033323F0030302EB411043EAC44343F056
:10269000C043C0F8103B2B6803F00303012B09B2C1
:1026A0000ED1D2F8083802EB411013F4807FD0F835
:1026B000003B14BF43F0805343F00053C0F8003B8D
:1026C00002EB4112D2F8003B43F00443C2F8003B56
:1026D00030BD00002DE9F041244D6E6D06EB401336
:1026E0000446D3F8087BC3F8087B38070AD5D6F828
:1026F0001438190706D505EB84032146DB68284604
:102700005B689847FA072FD5D6F81438DB072BD526
:1027100005EB8403D968CCB98B69488A5E68B6FB3F
:10272000F0F200FB12628AB91868DA6890420DD2A2
:10273000121A83E81400202383F311880B482146E2
:10274000FFF78AFF84F31188BDE8F081012303FAC3
:1027500004F26B8923EA02036B81CB6823B1214623
:102760000248BDE8F0411847BDE8F081AC2C0020DC
:1027700000EB810370B5DD68436D6C692668E66027
:102780004A0156BB1A444FF40020C2F810092A68C7
:1027900002F00302012A0AB20ED1D3F8080803EBB3
:1027A000421410F4807FD4F8000914BF40F0805028
:1027B00040F00050C4F8000903EB4212D2F80009BF
:1027C00040F00440C2F80009D3F83408012202FAAC
:1027D00001F10143C3F8341870BD19B9402E84BF0C
:1027E0004020206020682E8A841940F00050013C6F
:1027F0001A44B4FBF6F440EAC440C6E7F8B5044610
:102800001E48456D05EB4413D3F80869C3F8086901
:10281000F10717D5D5F81038DA0713D500EB840384
:10282000D9684B691F68DA68974218D2D21B002713
:102830001A605F60202383F311882146FFF798FF19
:1028400087F31188330617D5D5F834280123A34020
:10285000134211D02046BDE8F840FFF71FBD012309
:1028600003FA04F2038923EA020303818B68002B35
:10287000E8D021469847E5E7F8BD00BFAC2C002022
:1028800097482DE9F84F456D6E69AB691E4016F407
:10289000805F6E61044605D0FEF700FDBDE8F84F8D
:1028A000FFF780BC002E12DAD5F8003E8C489B075B
:1028B0001EBFD5F8003E23F00303C5F8003ED5F84F
:1028C000043823F00103C5F80438FEF715FD370579
:1028D00005D58348FFF7AEFC8148FEF7FDFCB00448
:1028E0000CD5D5F8083813F0060FEB6823F47053B5
:1028F0000CBF43F4105343F4A053EB60310704D5ED
:102900006368DB680BB176489847F2025AD4B30289
:102910000CD5D4F85480DFF8C8A100274FF0010986
:10292000A36D9B68F9B28B4280F08780F70619D5BA
:10293000616D0A6AC2F30A1702F00F0302F4F01283
:10294000B2F5802F00F0A180B2F5402F0AD104EB40
:10295000830301F58051DB68186A00231A469F4201
:1029600040F087803003D5F8184813D5E10302D52D
:102970000020FFF7AFFEA20302D50120FFF7AAFE59
:10298000630302D50220FFF7A5FE270302D503202B
:10299000FFF7A0FE750381D5E00702D50020FFF701
:1029A0002DFFA10702D50120FFF728FF620702D5FE
:1029B0000220FFF723FF23077FF570AF0320FFF707
:1029C0001DFF6BE7D4F85480DFF814A100274FF007
:1029D0000109A36D9B685FFA87FB5B4597D308EB02
:1029E0004B13D3F8002902F44022B2F5802F22D1F4
:1029F000D3F80029002A1EDAD3F8002942F09042C9
:102A0000C3F80029D3F80029002AFBDB5946606D82
:102A1000FFF73AFC228909FA0BF322EA0303238128
:102A200004EB8B03DB689B6813B15946504698470B
:102A30005846FFF733FC0137CBE708EB4112D2F8D9
:102A4000003B03F44023B3F5802F10D1D2F8003BB4
:102A5000002B0CDA628909FA01F322EA030363818D
:102A600004EB8103DB68DB680BB150469847013704
:102A700056E79C0708BF0A68072B98BF027003F14E
:102A800001039CBF120A013069E7023304EB8302A1
:102A900001F58051526890690268D0F808C040681A
:102AA000A2EB000E0022104697420AD104EB8304E9
:102AB00063689B699A683A449A605A6817445F60F1
:102AC00050E712F0030F08BF0868964588BF8CF8DE
:102AD000000002F1010284BF000A0CF1010CE3E7DF
:102AE000AC2C0020436D03EB4111D1F8003B43F4C3
:102AF0000013C1F8003B7047436D03EB4111D1F85F
:102B0000003943F40013C1F800397047436D03EBFB
:102B10004111D1F8003B23F40013C1F8003B70478A
:102B2000436D03EB4111D1F8003923F40013C1F8D0
:102B30000039704700F1604300F01F02400903F5BF
:102B4000614309018000C9B200F1604083F80013BD
:102B500000F5614001239340C0F880310360704765
:102B600030B5039C0172043304FB0325C361049B4D
:102B700003630021059B00604060C1604261026107
:102B80008561046242628162C162436330BD0000BC
:102B90000022416A41610161C2608262C2626FF0DB
:102BA0000101FEF7F7BE000003694269934203D1B9
:102BB000C2680AB100207047181D70470369196088
:102BC000C2680132C260C2691344826903619342E0
:102BD00024BF436A03610021FEF7D0BE38B5044626
:102BE0000D46E3683BB16269131D1268A36213448A
:102BF000E362002038BD237A33B929462046FEF728
:102C0000ADFE0028EDDA38BD6FF00100FBE70000F3
:102C1000C368C269013BC36043691344826943616D
:102C2000934224BF436A436100238362036B03B171
:102C30001847704770B52023044683F31188866ACD
:102C40003EB9FFF7CBFF054618B186F31188284639
:102C500070BDA36AE26A13F8015BA362934202D3D8
:102C60002046FFF7D5FF002383F31188EFE700002C
:102C70002DE9F84F04460E4690469946202787F3E3
:102C800011880025AA46D4F828B0BBF1000F09D15D
:102C900049462046FFF7A2FF20B18BF31188284652
:102CA000BDE8F88FA16AE36AA8EB050B5B1A9B45A8
:102CB00028BF9B46BBF1400F1BD9334601F14002B0
:102CC00051F8040B43F8040B9142F9D1A36A403345
:102CD0004036A3624035A26AE36A9A4202D3204694
:102CE000FFF796FF8AF311884545D8D287F31188FC
:102CF000C9E730465A46FDF7B5FFA36A5B445E4418
:102D0000A3625D44E7E7000010B5029C0172043342
:102D100003FB0421C36100238362C362039B03633B
:102D2000049B00604060C460426102618161046292
:102D30004262436310BD0000026AC260426A42619F
:102D4000026100228262C2626FF00101FEF722BEC0
:102D5000436902699A4203D1C2680AB100207047F0
:102D6000184650F8043B0B6070470000C368C26906
:102D70000133C3604369134482694361934224BFB2
:102D8000436A43610021FEF7F9BD000038B50446EF
:102D90000D46E3683BB123691A1DA262E269134440
:102DA000E362002038BD237A33B929462046FEF776
:102DB000D5FD0028EDDA38BD6FF00100FBE700001B
:102DC00003691960C268013AC260C269134482692A
:102DD0000361934224BF436A036100238362036B50
:102DE00003B118477047000070B5202304460E4613
:102DF00083F31188856A35B91146FFF7C7FF10B113
:102E000085F3118870BDA36A1E70A36AE26A01335C
:102E10009342A36204D3E16920460439FFF7D0FF4F
:102E2000002080F3118870BD2DE9F84F04460D464F
:102E300091469A464FF0200888F311880026B34641
:102E4000A76A4FB951462046FFF7A0FF20B187F38C
:102E500011883046BDE8F88FA06AE76AA9EB06033F
:102E60003F1A9F4228BF1F46402F1BD905F1400340
:102E700055F8042B40F8042B9D42F9D1A36A403346
:102E8000A3624036A26AE36A9A4204D3E16920460B
:102E90000439FFF795FF8BF311884E45D9D288F39B
:102EA0001188CDE729463A46FDF7DCFEA36A3B448C
:102EB0003D44A3623E44E5E7026943699A4203D177
:102EC000C3681BB9184670470023FBE7836A002BD1
:102ED000F8D0043B9B1AF5D01360C368013BC36074
:102EE000C3691A44836902619A4224BF436A036139
:102EF000002383620123E5E700F090B84FF08043A0
:102F0000002258631A610222DA6070474FF0804352
:102F10000022DA60704700004FF08043586370472A
:102F20004FF08043586A70474B6843608B688360FA
:102F3000CB68C3600B6943614B6903628B69436271
:102F40000B6803607047000008B5224B22481A69DD
:102F500040F2FF110A431A611A6922F4FF7222F04B
:102F600001021A611A691A6B0A431A631A6D0A433D
:102F70001A651A4A1B6D1146FFF7D6FF184802F171
:102F80001C01FFF7D1FF174802F13801FFF7CCFF12
:102F9000154802F15401FFF7C7FF144802F1700110
:102FA000FFF7C2FF124802F18C01FFF7BDFF114885
:102FB00002F1A801FFF7B8FF0F4802F1C401FFF7C3
:102FC000B3FF0E4802F1E001FFF7AEFFBDE8084095
:102FD00000F0AAB800380240000002409436000811
:102FE0000004024000080240000C024000100240B1
:102FF0000014024000180240001C02400020024061
:1030000008B500F007FAFEF731FCFFF785F8BDE8D8
:103010000840FEF75BBE000070470000104B1A6CC2
:1030200042F001021A641A6E42F001021A660D4A59
:103030001B6E936843F0010393604FF0804353226B
:103040009A624FF0FF32DA6200229A615A63DA60C4
:103050005A6001225A6108211A601C20FFF76ABDDC
:1030600000380240002004E04FF0804208B51369A8
:10307000D1680B40D9B2C9439B07116107D5202302
:1030800083F31188FEF712FC002383F3118808BD37
:1030900008B5FFF7E9FFBDE80840FFF783B8000077
:1030A0001F4B1A696FEAC2526FEAD2521A611A694B
:1030B000C2F308021A614FF0FF301A695A69586169
:1030C00000215A6959615A691A6A62F080521A627B
:1030D0001A6A02F080521A621A6A5A6A58625A6A66
:1030E00059625A6A1A6C42F080521A641A6E42F09F
:1030F00080521A661A6E0B4A106840F48070106095
:10310000186F00F44070B0F5007F1EBF4FF48030A0
:1031100018671967536823F40073536000F05AB9B5
:103120000038024000700040334B4FF080521A6468
:10313000324A4FF4404111601A6842F001021A60AD
:103140001A689207FCD59A6822F003029A602A4B0B
:1031500019469A6812F00C02FBD1186800F0F900C9
:1031600018609A601A6842F480321A600B689B03F8
:10317000FCD54B6F43F001034B671F4B5A6F900711
:10318000FCD51F4A5A601A6842F080721A601B4AC6
:1031900053685904FCD5184B1A689201FCD5194A9A
:1031A0009A60194B1A68194B9A42194B21D1194A46
:1031B0001168194A91421CD140F205121A60144A52
:1031C000136803F00F03052BFAD10B4B9A6842F0FA
:1031D00002029A609A6802F00C02082AFAD15A6C2C
:1031E00042F480425A645A6E42F480425A665B6EE0
:1031F000704740F20572E1E700380240007000407D
:103200000854400700948838002004E0116400202E
:10321000003C024000ED00E041C20F41084A08B501
:10322000536911680B4003F00103536123B1054A50
:1032300013680BB150689847BDE80840FEF7B2BF6D
:10324000003C0140242D0020084A08B5536911684C
:103250000B4003F00203536123B1054A93680BB19D
:10326000D0689847BDE80840FEF79CBF003C01408D
:10327000242D0020084A08B5536911680B4003F05B
:103280000403536123B1054A13690BB15069984790
:10329000BDE80840FEF786BF003C0140242D002019
:1032A000084A08B5536911680B4003F008035361DD
:1032B00023B1054A93690BB1D0699847BDE808402E
:1032C000FEF770BF003C0140242D0020084A08B5DD
:1032D000536911680B4003F01003536123B1054A91
:1032E000136A0BB1506A9847BDE80840FEF75ABF11
:1032F000003C0140242D0020174B10B55C691A6872
:10330000144004F478725A61A30604D5134A936AF0
:103310000BB1D06A9847600604D5104A136B0BB105
:10332000506B9847210604D50C4A936B0BB1D06BB8
:103330009847E20504D5094A136C0BB1506C9847C5
:10334000A30504D5054A936C0BB1D06C9847BDE832
:103350001040FEF727BF00BF003C0140242D002095
:103360001A4B10B55C691A68144004F47C425A6127
:10337000620504D5164A136D0BB1506D98472305AD
:1033800004D5134A936D0BB1D06D9847E00404D572
:103390000F4A136E0BB1506E9847A10404D50C4A26
:1033A000936E0BB1D06E9847620404D5084A136F30
:1033B0000BB1506F9847230404D5054A936F0BB1A6
:1033C000D06F9847BDE81040FEF7ECBE003C0140CE
:1033D000242D0020062108B50846FFF7ABFB062187
:1033E0000720FFF7A7FB06210820FFF7A3FB062114
:1033F0000920FFF79FFB06210A20FFF79BFB062110
:103400001720FFF797FB06212820BDE80840FFF7AB
:1034100091BB000008B5FFF743FE00F00BF8FDF785
:10342000CFFEFDF7A3FDFFF7F7FDBDE80840FFF76E
:1034300063BD0000002304491A465A50C8180833D7
:10344000802B4260F9D17047242D0020034611F8EB
:10345000012B03F8012B002AF9D170471210121327
:103460001211000053544D3332463F3F3F000000DD
:1034700000000000643400083F0000001304000056
:10348000A03400083F00000019040000AA3400081E
:103490003F00000021040000B43400083F00000099
:1034A00053544D3332463430780053544D33324602
:1034B0003432780053544D33324634343658580041
:1034C00000000000E50E0008D10E00080D0F0008F6
:1034D000F90E0008050F0008F10E0008DD0E0008C7
:1034E000C90E0008690F000800000000010000007C
:1034F000000000006D61696E0000000014350008D6
:10350000D823002050250020010000006918000881
:103510000000000069646C6500000000020000000B
:10352000000000001111000879110008400040005F
:10353000E8290020F8290020020000000000000017
:103540000300000000000000BD11000800000000A2
:1035500010000000082A0020000000000100000008
:1035600000000000AC2C00200101020041726475D3
:1035700050696C6F740025424F415244252D424CD6
:10358000002553455249414C250000006D1C0008A0
:10359000851B00081D1C0008011C000843000000DA
:1035A000A435000809024300020100C032090400EA
:1035B00000010202010005240010010524010001A0
:1035C000042402020524060001070582030800FF07
:1035D00009040100020A0000000705010240000082
:1035E000070581024000000012000000F0350008CD
:1035F00012011001020000400912415700020102AD
:10360000030100000403090425424F4152442500F0
:103610004D616D62614634303555532D493243005A
:1036200030313233343536373839414243444546F8
:1036300000000000004000000040000000400000CA
:103640000040000000000100000002000000020035
:103650000000020000000200000002000000020062
:1036600000000200000000000D130008ED15000826
:1036700099160008400040000C2D00200C2D002061
:10368000010000001C2D002080000000400100000F
:10369000030000000000800200000000AAAAAAAAFD
:1036A00000000000FFFF00000000000000A00A0072
:1036B0000000000000000000AAAAAAAA0000000062
:1036C000FFFF0000000000000000000000000050AC
:1036D00000000000AAAAAAAA00000000FF3F000004
:1036E00000000000000000000000000000000000DA
:1036F000AAAAAAAA00000000FFFF00000000000024
:10370000000000000000000000000000AAAAAAAA11
:1037100000000000FFFF00000000000000000000AB
:103720000000000000000000AAAAAAAA00000000F1
:10373000FFFF00000000000000000000000000008B
:1037400000000000AAAAAAAA00000000FFFF0000D3
:103750000000000000000000000000000000000069
:103760000A0000000000000003000000000000004C
:103770000000000000000000000000000000000049
:103780000000000000000000000000000000000039
:103790000E0400000000000000400F00FF00960033
:1037A000000000080096000000000800040000006F
:1037B00004360008000000000000000000000000C7
:0C37C000000000000000000000000000FD
:00000001FF
